:020000020000FC
:1000000099CE00000000000020C0C1C18EC00000D9
:10001000000098C000000000000000000203040679
:10002000080C10182030406080000406080C1018DE
:100030002030406080A0C0000003070F1F000D0D9E
:100040000403060D0503030202004FB662FD0CC057
:10005000552041F00994C52DC095089483FDC7959E
:10006000C4BD64604FBE1895C0916400089483FDC0
:10007000C795C4BD6B7FC0916400CF3F09F41EC01B
:1000800070FF1AC082FD05C04FBE93989498959852
:10009000189576FD0EC064FD0CC0C091B100C0FD86
:1000A0009298C1FDC298C2FDC198CAEFC095CA9589
:1000B000F1F79398949895984FBE189524BCCC2747
:1000C000C064C8BF6460F8CFC6CF70FFC4CF64FD02
:1000D000C2CF939AC0CF70FFBECF64FDBCCF949ABD
:1000E000BACF70FFB8CF64FDB6CF959AB4CF929ACD
:1000F00070FFB1CF64FDAFCFC7E0CA95F1F7939A17
:10010000AACFC29A70FFA7CF64FDA5CFC7E0CA955A
:10011000F1F7949AA0CFC19A70FF9DCF64FD9BCF59
:10012000C7E0CA95F1F7959A96CF4FB6C9B7CF7E7B
:10013000C9BF6E7FCCB5CE0DDDB5DF1DDBBDCABD41
:100140004FBE18953FB68F7EA9B7A072A2118061ED
:10015000A9B7AF7DA9BFA9B7AE7FA9BF7894A09179
:100160006800AA2341F085FD2FC0A0916800AA95E0
:10017000A093680029C040E050E085FD15C0A6B3FB
:1001800096FDA095A0FD4FEFAEB5A06496FDAF7BA8
:10019000AEBDAA27A062A8BF8D7FA6B396FDA0958D
:1001A000A0FD5FEF451739F7A0E461FDA09368005B
:1001B00085FD03C0A0E4A093680040939600816091
:1001C000442311F02092990085FD0EC0A091690092
:1001D000AA2331F0A0916900AA95A093690004C0F8
:1001E0008061AA27A062A8BF80FF0AC0A0919600E4
:1001F0004A2F61FF8E7F85FD01C000C040936100E2
:100200004091B400443009F004C0A0916100A09373
:100210006300A0916000A395A093600059F0F8944A
:10022000A9B7A160A9BF84FF03C0A9B7A062A9BFF5
:100230003FBE1895A0917400A395A093740042E06E
:1002400050916800552329F085FF03C05A955093BB
:100250006800A0919600A13018F0209299000DC07E
:1002600020929A002092A300A0919900AF5FA093E2
:10027000990018F0AFEFA0939900B09061005091F1
:10028000B400523049F465FF91F0A2E3BA1678F059
:10029000A0918600A0936100533049F465FF39F0C6
:1002A000A2E3BA1620F0A091C000A0936100509183
:1002B00062005B1521F010F05A9501C053955093E0
:1002C00062004A95D1F65091A300539509F45A95CE
:1002D0005093A300A091A400AA95A093A40009F0B4
:1002E0004BC0A1E0A093A40048E0A091A500AA23E0
:1002F00081F145E0A091A5005A17F0F1A091A60068
:100300005A1728F441E0A3E0A093A40007C0A091ED
:10031000A7005A1718F441E04093A400D0909C0025
:10032000C0906300DC14A8F0A091B400A430D9F010
:1003300065FD0FC0C0929C00539521F0A091A500CF
:10034000A093A300A1E0A093A400ACE3A09362005B
:1003500013C0A0919C00A40F20F45FEF50939C0069
:1003600002C0A0939C00A0919C00AF3F29F4AFEF86
:10037000A0939A00A093A300F894A9B7A160A9BF85
:1003800084FF03C0A9B7A062A9BF3FBE18953FB6BE
:1003900046B557B58F7EA9B7A072A2118061A9B7E3
:1003A000AF7DA9BFA9B7AE7FA9BF789481FD25C055
:1003B000AEB5AF7B96FDA064AEBD8260A6B396FDE0
:1003C000A095A0FF05C040936500509366001FC133
:1003D000AEB5A06496FDAF7BAEBDAA27A062A8BF54
:1003E0008D7F85FF01C006C140E0A6B396FDA095B4
:1003F000A0FD00C140939600EFC0AEB5A06496FD8D
:10040000AF7BAEBD8D7F61FF72C0AEB5AF7B96FD99
:10041000A064AEBDAA27A062A8BF826040939100ED
:1004200050939200A0908F004A19B09090005B0901
:10043000BB24A22C4C38520518F42092950049C0D8
:10044000A091D400AA2359F1483C520528F4A0E118
:10045000BA2EAAE0AA2E23C04836A1E05A0728F4F3
:10046000A8E0BA2EAFE0AA2E1AC0403DA2E05A077B
:1004700028F4A4E0BA2EAEE1AA2E11C0403AA5E0BD
:100480005A0728F4A2E0BA2EACE3AA2E08C04839D5
:10049000A8E05A0720F4A1E0BA2EA8E7AA2EC42E9D
:1004A000A0919300CA1AD52EA0919400DA0ADD20FB
:1004B0002AF4AFEFC094D094CA1ADA0A20929500B9
:1004C000A8E0A210A0E0CA14DA0618F4A1E0A093F4
:1004D0009500409393005093940040919100509167
:1004E000920040938F005093900042E075C0A0911D
:1004F00065004A1BA09166005A0B94FD60C093FDF5
:100500005EC092FD5AC086FF03C0D52EC42E0CC01B
:100510005695479591FD51C05695479590FD4DC014
:10052000D52EC42ED694C79461FD19C0AC2DAC5104
:10053000AD2DA24008F005C0DD2089F4AC2DA85CEB
:1005400070F4A0916700A395AA2311F0A09367000F
:10055000AA3008F44FC02092960081604BC0A09151
:100560006700AA2319F0AA95A0936700A22C5091C6
:10057000BA0097FD02C0A090C800AAEFAA0EA22D53
:10058000A21DCA18DA0A4FB74170442319F040E09F
:1005900050E015C0AFEFCA16D20418F04FEF50E08C
:1005A0000EC0A091AC00CA9E412D000C441F50E02B
:1005B00008F012C04FEF50E00FC05695479594FFDA
:1005C00007C0552309F04FEFA42FA6954A0F521DDF
:1005D0004F3F520508F04FEF40939600816061FF56
:1005E00009C0AFE1A095A923AB299A2F8F7DBB202D
:1005F00009F48062A0E4A093680085FF03C0AAE02C
:10060000A093680061FD03C085FD01C08F7E85FD5C
:1006100003C0A0E2A0936900F894A9B7A160A9BFA4
:1006200084FF03C0A9B7A062A9BF3FBE189511E01F
:100630000AC013E008C01AE006C01EE104C014E6B8
:1006400002C018EC00C005E1BB27BA95F1F70A9586
:10065000D9F71A95C1F708952AE338E709C020E3CE
:100660003CE806C02AE234EB03C025E238EC00C0C7
:10067000B091AD00BA9509F4089512E0BB27C29A73
:10068000BA95F1F7949ABA95F1F79498BA95F1F76B
:10069000C298BA95F1F7123009F0939A123009F422
:1006A000959AB091AD00BA95F1F7123009F0939890
:1006B000123009F49598B7E8BA95F1F71A95F1F662
:1006C000022FB22FBA95F1F70A95D9F73A9581F62C
:1006D000C29A0895221B39E0001F3A9509F4089543
:1006E000221F211B18F4210F8894F6CF0894F4CF11
:1006F000622C722CB0E08894B395221F331FE0F770
:10070000379527958894912E802E020B130B10F4A9
:10071000192D082D10F4889401C00894661C771CCC
:10072000BA9571F7172D062D0895322D11232AF44D
:100730003A9500951095031B130BF894029F712CAA
:10074000002D129F912C802C7894780C172D921CE0
:10075000292DB4E06B2E2695179507956A94D9F745
:10076000332321F000951095031B130B089500917E
:10077000B400043009F474C0B0919600B95198F0F7
:10078000B72FB67081F465FD2BC005E09090C600D0
:10079000B92DBA9521F00AE0BA9509F002E1B091BD
:1007A0007B00B01BE0F065FF0AC0B0919E00B093E3
:1007B0009C00BFEFB093A300B1E0B093A400B09150
:1007C0006100B093630020927E0020927F0020920F
:1007D000800020928100209282006F7D41C0606283
:1007E0009090C600B92DBA9579F4B0916200B09599
:1007F000BB1FBB1F1B2FB7950B2FB12FB170B3952C
:100800001B2FB02FBE7F25C0B92DBA95BA9581F4A4
:10081000B0916200B095BB1FBB1FBB1F1B2FB795CC
:100820000B2FB12FB370B3951B2FB02FBC7F14C00B
:10083000B0916200B095BB1FBB1FBB1FBB1F1B2F1E
:10084000B7950B2FB12FB770B395B3951B2FB02F62
:10085000B87FB0540B2F120900937E0010937F00D5
:10086000089510917B00169500917A000795B0913C
:100870007E00B01B0B2FB0917F00B10B1B2F28F413
:100880000038BFEF1B0740F009C00F37120508F40E
:1008900005C00FE710E002C000E81FEF00938300DF
:1008A00010938400089500918300B09180000B0F95
:1008B00010918400B09181001B1F20E030918400D2
:1008C00033230AF42A95B09182002B1F1AF4203F9B
:1008D00040F00AC02F3008F407C00FEF1FEF2FE0E1
:1008E00003C000E010E020EF30916300B0919B0066
:1008F0003B1718F4323030F009C0B0918400BB23AC
:100900005AF004C0B0918400BB2332F400938000FD
:10091000109381002093820008952091D7000091C8
:100920008300000F10918400111FFFDE11232AF4B1
:100930000038BFEF1B0740F009C00F37120508F45D
:1009400005C00FE710E002C000E81FEF002352F0DF
:10095000B0916200B01B0B2F18F0013008F00AC0F4
:1009600001E008C000950F5FB09162000B0F08F026
:1009700001C00FEF0093850008952091D8000091E9
:10098000810010918200D1DE11232AF40130BFEFE3
:100990001B0740F009C00F3F120508F405C00FEF18
:1009A00010E002C001E01FEF112352F0B09185006A
:1009B000B01B0B2F18F0013008F00AC001E008C08E
:1009C00000950F5FB09185000B0F08F001C00FEF8D
:1009D0000093630008950FEF71FD1EC0B091D30026
:1009E000BB23D1F0B0917B00BB23B1F00FEF10918E
:1009F0007B0070DEF894B091730072FDB5E00B9F40
:100A0000112D002D7894112309F00FEFB0919E0065
:100A10000B1710F400919E0000939D000895009123
:100A20007A0010917B0000541140B0919D0010F4A9
:100A3000BA9501C0B39511F0B0939D000895FCD311
:100A4000B7E074FDB6E0B06CB7B9B6B1B068B064E9
:100A5000B6B9EDDDB7E074FDB6E0B06CB7B9B6B1CC
:100A6000B068B064B6B9B6B1B6FDFDCF04B115B18A
:100A7000B6B1BF77B6B939D42AEB2093A8002223A8
:100A800009F441C030E03093A900732E7694622EB1
:100A90006694620E731E262D372D0217130778F009
:100AA0008090A800BAEBB80DB093A8008090A90080
:100AB000B0E0B81DB093A900260D371DEECF809091
:100AC000A8009090A9001091A90016950091A80087
:100AD00007951695079523E0169507952A95E1F752
:100AE0002091B5002A9529F42092A8002092A9000F
:100AF0000AC02A9521F0800E911E2A95E1F7809276
:100B0000A8009092A90008952091B500B6B1B6FD55
:100B1000FBCF04B115B1B6B1BF77B6B9B091AA0099
:100B2000B395B093AA00B83060F12092AA00B091BA
:100B3000D200BB2321F1112329F0B091AB00BF3FBC
:100B400061F009C0B091AB000B1739F020F4BB2362
:100B500021F0BA9502C0B395E1F300919B00B093E8
:100B6000AB00B93B50F400ECBA3A38F400E8BB39BA
:100B700020F400E4BC3808F400E000939B007F7E82
:100B800008952130B1F00F3FB3E01B0790F4BAEBAA
:100B9000BB2379F0B091A8000B17B091A9001B07F7
:100BA00040F4B0919B00BB2359F0BA95B0939B00E1
:100BB00007C0B0919B00BF3F19F0B395B0939B0065
:100BC00000919B00B0916300B01B10F40091630092
:100BD000B0919C000B1750F000919C00B0919C00CC
:100BE000BF3F21F0B0919C00B0939B00502E00932A
:100BF0006400B091AA00B73009F47061089502E36F
:100C0000F894B091D9000B9F012D000C001F78942F
:100C1000B0919B000B1710F000919B0000936100B6
:100C200000936300502E0093640000939E0008958B
:100C300020927A00B0EFB0937B000895F8940CB541
:100C40001DB5209174007894309175006090760005
:100C50000093750010937600031B160971FD03C005
:100C600077FD80C028C07090770020937700270917
:100C7000222319F00FEF1FEF0EC0809078009090A4
:100C8000790030937800609279000091750010919E
:100C900076000819190920917A0030917B00369569
:100CA0002795020F131F10F40FEF1FEF00937A0028
:100CB00010937B002BC020917A0030917B0039018A
:100CC000B4E08B2EB2E09B2E343040F08A949A949C
:100CD000383020F072FD02C08A949A94769467941A
:100CE0008A94E1F726193709992021F0169507957E
:100CF0009A94E1F7200F311F20937A0030937B0004
:100D000028F43FEF30937A0030937B00323008F4C0
:100D1000706871FF02C0B3E00DC0B091C4000091D3
:100D20007100023838F0B395003A08F0B395B63048
:100D300008F0B5E09B2EB4E08B2E10917B00009163
:100D40007A0024E0169507952A95E1F7081912090B
:100D500028F0B02FB250B12FB20910F402E010E029
:100D6000980126C020917A0030917B003901769459
:100D700067946694669466942619320906950695DA
:100D8000200F321D20937A0030937B00323008F020
:100D90007F7704E0369527953695279526952695F5
:100DA000201B10F0223008F422E089019090C4004A
:100DB00060FDFECFE0908B00F0908C006160B9B7D1
:100DC000B061B9BF380177FD41C076946794009354
:100DD0008B0010938C00B92DB330E1F0B0FD04C04E
:100DE000060D171D930106C0000F111F02501209B6
:100DF00022E030E0B92DB33068F020938D003093BD
:100E00008E00009387001093880060928900709292
:100E10008A003AC000938D0010938E0020938700C3
:100E2000309388006092890070928A0071FF0DC033
:100E3000BFE0B0938D0020928E00B0938900209285
:100E40008A00B0938B0020928C001EC066940093A1
:100E50008B00B92DB33091F0B0FD03C0060D262DE7
:100E600003C0000F025022E0B92DB33038F02093B8
:100E70008D00009387006092890006C000938D006A
:100E8000209387006092890000917C0002FD03504E
:100E9000013049F495FD12C0B0B7B860B0BFB0E002
:100EA000B06CB7B90EC0023039F4B0B7B860B0BF9B
:100EB000B1E0B06CB7B905C095FDEECFB0B7B77F64
:100EC000B0BF0091A200000F10F4BBE60B27009307
:100ED000A20060FDFECFB2E0B0936E006160B9B7D2
:100EE000B061B9BFB72FB670D1F020917A003091C0
:100EF0007B00369527953695279571FF02C0B0E4A3
:100F00003B0FF8940CB51DB5020F131F1BBD0ABD96
:100F10006160B0E1B8BFB9B7B061B9BF7894089566
:100F2000686020927D0020E066FD20E206C06860D7
:100F300020927D0020E266FD20E001E011E077FDD7
:100F400011C0B72FB67009F0677F14E100917B00E4
:100F5000069509F403950F3008F00FE071FF02C009
:100F600004E114E160FD0FC0B0917D00BB2359F096
:100F700071FF06C0B0916E00BA95B0936E0011F487
:100F8000706251C0ABDFB0B73B2FB77FB0BFB8B115
:100F9000B0B733FDB860B0BFB0917D00B395B093EA
:100FA0007D00B8B177FD06C0B1E071FDB3E0BA9540
:100FB000F1F7B8B1B072B21709F02AC071FF05C0DD
:100FC0000395011708F00A95CDCF63FD05C0039581
:100FD000011708F0B2CFC6CF677FF8943CB56DB467
:100FE00070907A00B0917B00770CBB1F08F4BFEFC4
:100FF000770CBB1F08F4BFEF370D6B1E6BBC3ABDFF
:101000006160B0E1B8BFB9B7B061B9BF789495CFAE
:10101000B0916D00B13008F490CF63FD8ECF0A958A
:1010200009F0A0CF7F7D20918D0030918E00F89443
:10103000B0E1B8BF0CB51DB5020F131F1BBD0ABD33
:10104000E0908700F09088006160B9B7B061B9BFE7
:101050007894B72FB67039F0B0916D0072FFB395E8
:10106000B0936D0009C075FF07C066FD05C063FD44
:1010700003C0BF91BF9105C5089500E063FF01C0A3
:1010800001E0F89410917100B7E01B9F212D102D05
:101090007894200F269517952695179526951795E0
:1010A00010937100183718F4B8E7B09371000091ED
:1010B0007100B09172000B1720F0606193989498C2
:1010C000959860FDFECFE0908900F0908A00616005
:1010D000B9B7B061B9BF0895AC98B2E095FD0AC048
:1010E000F894B0937C00C29A929862FF01C0959ADE
:1010F0007894F9C0F894B0937C00C29AC19862FFCA
:1011000001C0939A7894EFC0AC9AB3E082FF24C0F8
:1011100095FD11C002E0F894B0937C00E1E8F0E0A6
:101120000093B1009598C19A62FF02C0949A01C0E1
:10113000C2987894D8C002E0F894B0937C00E1E8BB
:10114000F0E00093B1009398929A62FF02C0949AE3
:1011500001C0C2987894C7C095FD0BC0F894B093B5
:101160007C00EBE6F0E0959862FF01C0949A7894D9
:10117000BAC0F894B0937C00EBE6F0E0939862FF7D
:1011800001C0949A7894AFC0AC98B4E095FD0AC0C1
:10119000F894B0937C00929AC19862FF01C0949A2F
:1011A0007894A1C0F894B0937C00C19A929862FFA1
:1011B00001C0949A789497C0AC9AB5E082FF24C09D
:1011C00095FD11C001E0F894B0937C00E7E7F0E0F2
:1011D0000093B1009498C29A62FF02C0939A01C032
:1011E0009298789480C004E0F894B0937C00EBE887
:1011F000F0E00093B1009498C29A62FF02C0959A01
:1012000001C0C19878946FC095FD0BC0F894B0935D
:101210007C00E5E6F0E0949862FF01C0939A789430
:1012200062C0F894B0937C00E1E7F0E0949862FF2C
:1012300001C0959A789457C0AC98B6E095FD0AC065
:10124000F894B0937C00C19AC29862FF01C0939A4F
:10125000789449C0F894B0937C00929AC29862FF47
:1012600001C0959A78943FC0AC9AB1E082FF24C047
:1012700095FD11C004E0F894B0937C00EBE8F0E039
:101280000093B1009398929A62FF02C0959A01C0B0
:10129000C198789428C001E0F894B0937C00E7E707
:1012A000F0E00093B1009598C19A62FF02C0939A52
:1012B00001C09298789417C095FD0BC0F894B09334
:1012C0007C00E1E7F0E0939862FF01C0959A789482
:1012D0000AC0F894B0937C00E5E6F0E0959862FFD0
:1012E00001C0939A78946F7E089524E630E0F90166
:1012F0002092B100939894989598929AC29AC19A24
:101300006B7F0895A2EBB0E007E00D9307E00D932B
:1013100001E00D9304E00D930FEF0D930D9309E0A1
:101320000D9302E00D9301E00D9301E00D93AEEB00
:10133000B0E001E00D9300E00D9304EB0D930FEF8F
:101340000D930D930D9303E00D930FEF0D9301E0BB
:101350000D930FEF0D9305E20D9300ED0D9308E74C
:101360000D9308EC0D9304E00D930FEF0D9301E046
:101370000D9300E00D930AE70D930AE00D9300E052
:101380000D9301E00D9300E00D930FEF0D9300E03E
:101390000D9308952091B9008B7F233009F4846068
:1013A000B091BA009F7DB1FD90629F7BB091BB0070
:1013B000B1FD9064223011F0886001C0877F0895EC
:1013C0000A95E00FF21DB4910895ECE1F0E0009170
:1013D000B200F6DFB093D700ECE1F0E00091B3008B
:1013E000EFDFB093D800EAE2F0E00091B800E8DF68
:1013F000B093D9000091D100002319F42092A500E8
:1014000013C0013108F001E1B02FB00FB00FB0935D
:10141000A5001B2FB10FB10FB00FB093A600B10FF5
:10142000B00FB00FB093A7000091B800023008F4DD
:1014300002E000937300B091CE000FEFB23009F4D8
:1014400000EAB33009F402E800937200E8E3F0E048
:101450000091D500B5DFB093A000089508952091C4
:10146000C8003091C900B091BA00B33009F43E50C1
:1014700097FF02C020E03FEFB32FB21B6B2EB25894
:1014800010F4B2E86B2E00E00395609EB12DBD57BD
:10149000D8F30093AC0008959068E1DFCED8CDD8A2
:1014A00020E030E0B0E16B2EC4D8B09196002B0F55
:1014B000321D6A94C9F7B4E036952795BA95E1F7DD
:1014C000822E9F77CCDF0895F894E3E0F0E0B9E056
:1014D000B7BFB491B078C1F3F894A895B1B5B8612D
:1014E000B1BDB0E0B1BDB4E0BEBFBFE5BDBFFDDE84
:1014F000B6E0B8BBB6E1B7BBB8E0B5BBBCE1B4BBC6
:10150000B4E0B2BBBCE3B1BB2224A0E0B0E02D92BA
:10151000AA31E9F7A0E6B0E00FEF2D920A95E9F7BE
:10152000B1E0B093A200EEDEEDD2B7E0B06CB7B997
:10153000B6B1B460B068B6B90091CA000093AD000E
:10154000B1E0B0936A00F8947CD886D876D887D872
:1015500074D888D872D865D374D873D870D8F894F2
:101560000AEF1AEFA6B396FDA095A0FF1FC01A952B
:10157000C9F70A95B1F7E0E0FCE1B591B43E39F462
:10158000B591B03E21F4B591BF3F09F40CC0E0E045
:10159000F395F395B591B83F49F4B591B43931F469
:1015A000B591BA3A19F4EE27F6950994F3DE0DDFFA
:1015B00055DF55DF0091CA000093AD0096DEB2E022
:1015C000B3BFB2E0BEBDB2E0B5BDB1E5B8BFB9BF13
:1015D000B0B70B2FB77FB0BFB8B1B0B703FDB860DD
:1015E000B0BF25D878942BDA20927000BEB5B064D5
:1015F00096FDBF7BBEBDB9B7B062B9BFBB27B062B5
:10160000B8BF8D7F1ED8626033E02CE0B0919500AA
:10161000BB2321F42CE03A9509F4A1CF0ED880FF2A
:101620009ECF8E7FB0919600B23078F3B92FBF7104
:101630000091980000939700B0939800B01729F795
:101640002A9521F76D7FBEB5B06496FDBF7BBEBD08
:10165000BB27B062B8BF8D7FB091D400BB2321F40B
:101660008062B92FB0709B2F8F7B20926700E7D7E5
:1016700085FF05C0B0916700BA3008F08064D9D703
:1016800002E085FF01C000E0B0919600B017B8F30A
:10169000F894E2D7E1D7E0D77894D3D720928600A8
:1016A000C8D7B091BE00B13008F478C0B0916A00DC
:1016B000B13008F473C085FD18C0B0919600BF3FEB
:1016C00008F46CC0F894D1D77894B9D7B09196004B
:1016D000B130C0F7F894C0D7AED7BED77894AFD7A3
:1016E000B0919600BF3FB0F3CEC2B8E09B2E906899
:1016F000F894B5DE7894A3D7F8949F77B0DE809005
:101700009600B0919600BF37789408F44FC08FD7F9
:10171000F894ABD778949A9451F7BEDEB82DB550B3
:10172000B093C9008ED7F89481D27894BAE09B2EFA
:101730009068F89494DE789482D7F8949F778FDE3F
:1017400080909600B0919600BF37789478F76FD765
:10175000F89482D770D780D778949A9449F79CDE12
:10176000B82DBB5FB093C8000B2F1091C900125861
:1017700010F0100B20F4B2E80B0F0093C90061D7F2
:10178000F894EDD162D278945AD7F89468DE7894C0
:10179000B0919600BF3F08F48ECF75C200919600BD
:1017A000B09186000B1710F00093860048D701E037
:1017B000B091BA00B35009F405E0B0919600B017AB
:1017C00008F06ECFF89451D750D74FD7789439D7C7
:1017D00020926A0020926B0020926C00B0916B0006
:1017E000B395B0936B00BF3F71F5B0916C00B395AA
:1017F000B0936C00B091CC0009E1BA9559F002E3C6
:10180000BA9541F00DE7BA9529F00AEFBA9511F0B3
:1018100020926C00B0916C00B017A8F066DD07D77D
:10182000B0916C00BA95B0936C0020926B00B091AF
:10183000CB00B093AD00F89418D77894B091CA005B
:10184000B093AD00FCD6F7D6B0916800BB2319F475
:1018500085FF01C084CE01E085FD01C006E0B091A6
:101860009600B01708F4BACFEAD6B0916800BB234F
:1018700009F475CEF89439DD20926100209262005F
:1018800020926300522C209264002092A100789450
:10189000B091B700BB0FB0939F0020927E002092C2
:1018A0007F0020928000209281002092820020926E
:1018B000AA0060E070E020927100B8E0B093AA0046
:1018C0007061B5D6B7E074FDB6E0B06CB7B9B6B12B
:1018D000B068B064B6B9B6B1B6FDFDCF04B115B10C
:1018E000B6B1BF77B6B9112309F00FEF0093AB0083
:1018F0000BD9B8E0B093AA0070614CDDF894BFEF4B
:10190000B0939B007CD9B0916100B0939B00B093E1
:101910009C00B0939D007894B1E0B0936100B093C7
:1019200063005B2EB0936400B093A400B0919A0062
:10193000B093A300B091BA00B33019F49F7D87FD36
:1019400090627160726020926D0076DC8DDC70D9DF
:1019500075D96ED973D96CD9EADA09D78EDBBCDBBD
:101960006DD9DEDA65FD7DD777FF35D877FD57D89D
:1019700084DBCADB63D9DBDA65FD95D77EDB04DC6B
:101980005DD9CEDA65FDC9D778DB16DC57D9CFDA59
:1019900065FDF3D772DB50DC51D9C2DAB7E074FDD4
:1019A000B6E0B06CB7B9B6B1B068B064B6B965DBD3
:1019B0005BDC44D9A9D871FF1EC0B0919E00B093E2
:1019C0009B00B0939C00B0919A00B093A300B1E04B
:1019D000B093A40018E12CE0B0916D00B11728F08D
:1019E0007D7F746020936F0006C0B0919600B13087
:1019F00008F0B2CF50C072FF15C066FD13C0B091A1
:101A00006F00BA9519F47B7F7860A6CFB0936F0012
:101A1000B0919600B13008F09FCFB091BA00B330CA
:101A200009F039C020927000B0919900B13058F09F
:101A3000B0919E00B0939C00B0919A00B093A30027
:101A4000B1E0B093A400B09199000AEF1091D600D4
:101A5000112309F003E0B01708F01DC085FF04C092
:101A6000B0916800BB23B9F000EF66FF05C0B091EC
:101A70009E00B0939B0000E2B0917B00B01708F489
:101A80006BCFB0917000B395B0937000B091960099
:101A9000BB2309F002C020927000F89426DC8090ED
:101AA000B900B2E0B093B90075DC8092B900209221
:101AB00061002092620020926300522C2092640008
:101AC00020929F0060E070E07894B9D50EDC009120
:101AD000D600002319F0939A949A959AB7E0B06CC7
:101AE000B7B9B6B1B460B068B6B985FF05C0B091FA
:101AF0006800BB2309F433CDB091BF00B13008F0CA
:101B0000BECD68CEEDE0F0E023D0053A09F01BC071
:101B1000EEE0F0E01DD00A3509F015C03AE0A2EB86
:101B2000B0E0E3E0F0E014D00D9331963A95D9F7A8
:101B300039E1AEEBB0E0EFE0F0E00AD00D93319682
:101B40003A95D9F702C0DEDB0AD0E8E2F0E008956A
:101B5000E199FECFEEBBFFBBE09A0DB308951ED016
:101B60003AE0A2EBB0E0E3E0F0E00D910FD0319667
:101B70003A95D9F739E1AEEBB0E0EFE0F0E00D9146
:101B800005D031963A95D9F712D00895E199FECF54
:101B90000DBBEEBBFFBBE29AE19A0895EDE0F0E0E9
:101BA0000FEFF4DFEEE0F0E00FEFF0DF0895EDE08F
:101BB000F0E005EAEBDFEEE0F0E00AE5E7DF0895AC
:101BC0003091AE000091AF00313011F40093B200BB
:101BD000323011F40093B300333011F40093B400A9
:101BE000343011F40093C600353011F40093B50081
:101BF000363011F40093B800373011F40093C4006C
:101C0000383011F40093B900393011F40093CE004C
:101C10003A3011F40093BA003B3011F40093BB004A
:101C2000089525E00ED52A95E9F7089515D517D51D
:101C300019D51BD500D510D512D514D516D5FBD482
:101C40000BD50DD50FD511D508950FD50BD507D5CB
:101C500003D5F1D40AD506D502D5FED4ECD405D5EA
:101C600001D5FDD4F9D408958090AE009090AF00D6
:101C7000F3D4F2D4F1D4DFD48A94D1F7F6D4DBD400
:101C80009A94E1F70895F894D1DF7894CADFC9DF18
:101C9000B1E0B093AE00B1E0B093AF002092B000DD
:101CA000F894E2DF7894B5E06B2E70909600C9D47A
:101CB000B09196007B16C9F7B13018F0BF3F40F1E4
:101CC00007C07EDFF8944BDFB1DFB8E0B1BDA9DF1C
:101CD0006A9459F7B091B000B395B093B000B330A7
:101CE00008F4DECF9EDFB091AF00B395B093AF00A4
:101CF000F894B091AE00BA95EEE3F0E0EB0FF21D70
:101D0000049178940395B091AF00B01708F4C6CF52
:101D100088DF87DFB091AE00B395B093AE00B0918D
:101D2000AE00BC3008F4B7CFEDDAF89418DFB8E0B5
:061D3000B1BD77DFC9CB55
:00000001FF
